:100000000C943D010C945A010C945A010C945A0121
:100010000C945A010C945A010C945A010C945A01F4
:100020000C945A010C945A010C94A5190C94771A4B
:100030000C94CA140C945A010C945A010C945A0151
:100040000C945A010C945A010C945A010C945A01C4
:100050000C945A010C9452150C945A010C945A01A8
:100060000C945A010C945A010C945A010C945A01A4
:100070000C945A010C945A010C945A010C945A0194
:100080000C945A010C945A010C945A010C945A0184
:100090000C945A010C945A010C945A010C945A0174
:1000A0000C945A010C945A010C945A01F903F90367
:1000B000250425048D04B805B805B805AB0444052E
:1000C00055055505E41A0B1B031C0B1B031C571B82
:1000D0007A1B031CD11BE01B2B0014001A00080024
:1000E000150017001C0018000C00120013002A0055
:1000F000390004001600070009000A000B000D007B
:100100000E000F0000003400E10038001D001B004D
:100110000600190005001100100036003700E50048
:10012000E000E300E20000002A00000028002C00AC
:100130000000E6000151E40029001E001F0020001D
:1001400021002200230024002500260027002D0086
:10015000A900010001000100010001005000510050
:1001600052004F0000002800AA0001000100010019
:1001700001000100010001002D002E0038000100E7
:100180000100010001000000010000000100010069
:1001900000000100010001000E036A0075006C0000
:1001A00069006500740000000C036E0061006300CC
:1001B0006C00790000000403090409023B000201FD
:1001C00000A0FA0904000001030101000921110146
:1001D0000001224000070581030800010904010015
:1001E000010300000009211101000122320007056E
:1001F00082032000011201000200000008626B6906
:100200004001000102000105010980A101850319D7
:10021000012AB700150126B700950175108100C0AD
:10022000050C0901A101850419012AA00215012666
:10023000A002950175108100C005010906A1010504
:100240000719E029E7150025019508750181029538
:1002500001750881010507190029FF150026FF0017
:100260009506750881000508190129059505750190
:100270009102950175039101C00011241FBECFEFBB
:10028000DAE0DEBFCDBF11E0A0E0B1E0ECE1F9E3E0
:1002900002C005900D92A438B107D9F722E0A4E876
:1002A000B1E001C01D92AA34B207E1F70E94AA1181
:1002B0000C948C1C0C94000081E0089581E008955A
:1002C0000C945E0108950C9462011F93CF93DF9309
:1002D00000D000D01F92CDB7DEB749835A836B831D
:1002E0003091870189819A81311114C0662359F0B8
:1002F000222349F00E94F107182F682F89819A81E3
:100300000E949A0703C00E94C507182F69817A814D
:10031000812F04C00E94F10769817A810F900F90AC
:100320000F900F900F90DF91CF911F910C94150FAC
:10033000FC01262F408151816281738184810C945C
:10034000650181E00895CF93DF93EC0160E00E94A6
:100350009801BE01DF91CF910C9463010C945B1066
:100360000C94571008950E9444060E94B2012FEF8A
:1003700084E39CE0215080409040E1F700C0000001
:100380000C9478150F931F93CF93DF938C0161E04A
:100390000E949801EC01B8010E9460018823F1F1EC
:1003A000B801CE010E94A3138823C1F1B801CE0188
:1003B0000E94B711882391F1B801CE010E94FF126B
:1003C000882361F1F8018281882309F1CB358DE51D
:1003D000D807C1F050F4C115FCE5DF0781F0CF3D2F
:1003E000DC45A9F40E94280D19C0CC35EDE5DE07E7
:1003F00061F0CD35DD4559F40E946B0C08C00E94B8
:10040000B3010CC00E94740C02C00E94770CC8019A
:10041000DF91CF911F910F910C945C0180E0DF91EF
:10042000CF911F910F9108950E94AC140C942D024E
:100430000E9430020C94B21408950C941C0281E0C6
:1004400008950C941F020895CF93C82F0E941D0297
:100450008C2F0E942102CF91089580E00C942402F9
:100460000E94FF130C9424020E94FF1390918601B6
:10047000891721F0809386010C9424020895CF936C
:10048000DF93CDB7DEB72B970FB6F894DEBF0FBE64
:10049000CDBF4F83588769877A878B8761110E9408
:1004A000B70B9E012F5F3F4F86E0F90111928A95AD
:1004B000E9F785E0FE013796D90101900D928A9502
:1004C000E1F789819A814C815D81452B31F09F3F15
:1004D00031F491E08F3F19F403C091E001C090E046
:1004E00090FF09C049815A816B817C818D819E81F9
:1004F0000E94D80A05C0C9010E94A1018111F2CF52
:100500002B960FB6F894DEBF0FBECDBFDF91CF9113
:100510000895FC01808191810E9433080895CF9352
:10052000882309F49CC0C82F8238C1F40E94FF13AD
:1005300081FD95C069E380910201909103010E94C1
:1005400084140E94D90B2FEF81EE94E0215080405B
:100550009040E1F700C0000069E319C0833801F55D
:100560000E94FF1380FD7BC063E5809102019091A2
:1005700003010E9484140E94D90B2FEF81EE94E0B6
:10058000215080409040E1F700C0000063E5809179
:100590000201909103010E948614CF910C94D90B13
:1005A0008438C1F40E94FF1382FD59C067E4809132
:1005B0000201909103010E9484140E94D90B2FEF35
:1005C00081EE94E0215080409040E1F700C00000AF
:1005D00067E4DDCF8CEF8C0F813AD0F46C2F8091E3
:1005E0000201909103010E944E14882349F06C2F60
:1005F00080910201909103010E9486140E94D90B00
:100600006C2F80910201909103010E948414C5CF48
:1006100080E28C0F883048F4C77081E001C0880FF9
:10062000CA95EAF70E949A0BB8CFEBE5EC0FE330DE
:1006300040F4F0E0E15CFE4F808190E0CF910C94BB
:100640001614C85AC73158F4EC2FF0E0EE0FFF1F14
:10065000EF5EFE4F80819181CF910C942C14CF914D
:100660000895882309F45BC0682F823879F40E94CA
:10067000FF1381FF54C069E380910201909103014F
:100680000E9484140E94D90B69E310C08338B1F42E
:100690000E94FF1380FF43C063E5809102019091A7
:1006A00003010E9484140E94D90B63E5809102012A
:1006B000909103010E9486140C94D90B843879F42C
:1006C0000E94FF1382FF2BC067E48091020190918A
:1006D00003010E9484140E94D90B67E4E7CF8CEFDA
:1006E000860F813A18F380E2860F883048F46770ED
:1006F00081E001C0880F6A95EAF70E94A00BDCCF69
:100700008BE5860F833020F480E090E00C94161483
:10071000685A673120F480E090E00C942C1408951E
:100720001F93CF93DF93182FEB010E948F02209726
:1007300041F08FE99FE00197F1F700C00000219799
:10074000F6CF812FDF91CF911F910C943103893324
:1007500019F060E070E002C060E570E00C94900376
:10076000882321F00E949A0B0C94D90B08958823BA
:1007700021F00E94A00B0C94D90B0895CF92DF9228
:10078000EF92FF920F931F93CF93DF937C01D62FAD
:10079000C72FFC011281058102950F700E94900BFA
:1007A0008823B9F01123A9F08C2F807F803421F0A9
:1007B00080E28D0F883068F08091280282FD09C0A8
:1007C00082E00E94390C0E94900B91E0D82ED9262D
:1007D00001C0D12CCC2EC2948FE0C8228C2D90E089
:1007E0008C30910508F0C4C1FC01EA5AFF4F0C940B
:1007F000371C8C2F807FCF70882311F0C295C07F6B
:10080000112399F0CC2309F49FC180E28D0F883029
:1008100010F0D11104C08C2F0E949A0B03C08C2FB2
:100820000E94AA0B0E94D90B8FC18D2F0E94310309
:10083000CC2309F49DC180E28D0F883038F1DD238F
:1008400029F18C2F0E94B00B24C08C2F807FCF7099
:10085000803211F0C295C07FDD2319F0D130A1F1B3
:100860003DC08091280282FF17C0112349F0CC239C
:1008700029F08C2F0E949A0B0E94D90B80E065C151
:1008800080E00E943103CC2309F472C18C2F0E94B6
:10089000A00B0E94D90B6CC1112371F0002341F011
:1008A000013031F40E94BA0B8C2B0E94C20B60C144
:1008B0000E94BA0B8C2B1DC0002319F0013009F4E3
:1008C00057C10E94CF0B25C0112321F0063008F03C
:1008D0004FC10EC0053008F04BC11BC0112361F0A1
:1008E000002331F0F701858180FF2EC18F70858351
:1008F0008C2F0E94B0033CC1002359F0D93309F07A
:1009000034C1FFEF07EE13E0F15000401040E1F773
:100910002AC18C2F0E94B7032BC18C2F86958695F8
:10092000837019F0813061F023C1112321F08D2FE4
:100930009C2F937002C080E090E00E94161420C1AA
:10094000112321F08D2F9C2F937002C080E090E046
:100950000E942C1415C18C2F837009F047C011110F
:100960000BC12D2F229526952770220F220F6D2F58
:100970006F70862F90E0A0E0B0E0022E04C0880FD8
:10098000991FAA1FBB1F0A94D2F7D4FF10C04FE0D3
:1009900050E060E070E004C0440F551F661F771FF1
:1009A0002A95D2F7409550956095709503C040E028
:1009B00050E0BA01C695C695C3708A019B01082B09
:1009C000192B2A2B3B2BC901B801C23049F058F42E
:1009D000C13019F00E94B006CFC00E949E06CCC064
:1009E0000E94C206C9C00E949C06C6C0112319F00D
:1009F0008C2F817001C08695882309F4BDC02D2FEE
:100A0000229526952770220F220F6D2F6F70862F4B
:100A100090E0A0E0B0E0022E04C0880F991FAA1F4A
:100A2000BB1F0A94D2F7D4FF10C04FE050E060E043
:100A300070E004C0440F551F661F771F2A95D2F738
:100A4000409550956095709503C040E050E0BA0124
:100A5000C695C695C3708A019B01082B192B2A2BBA
:100A60003B2BC901B801C23049F058F4C13019F02C
:100A70000E94750781C00E9463077EC00E9487079D
:100A80007BC00E94D60678C0CF70112339F08C2F1E
:100A90000E94FC068D2F0E94B0036EC08D2F0E9415
:100AA000B7038C2F0E941D0767C0D23F21F128F4A5
:100AB000D03F41F0D13FC1F043C0D33F19F1D43F03
:100AC00079F03EC0112341F0053008F051C08C2F61
:100AD0008F710E9442074CC0063008F049C0F7CF22
:100AE0008091280282FF18C0112339F08C2F8F715A
:100AF0000E94FC063DC01123C9F38C2F8F710E9408
:100B00001D0736C0112329F08C2F8F710E94E70634
:100B10002FC00E94E2062CC0112349F0CF718C2F08
:100B20000E94FC0663E08C2F0E941E0C21C081E015
:100B30000E94390C0230E0F082E00E94390C18C0AB
:100B4000112331F0002391F28D2F0E948F0210C0EB
:100B5000002399F2D93349F41FEF27EE33E0115007
:100B600020403040E1F700C000008D2F0E9431038B
:100B700088EF8C0D843020F40E94FF130E94240221
:100B8000DD20C9F00E948C0B80FD15C0F701128298
:100B90000E94860B0E94FC06C7010E94FC050E9471
:100BA000860BDF91CF911F910F91FF90EF90DF9017
:100BB000CF900C941D07DF91CF911F910F91FF9063
:100BC000EF90DF90CF9008950F931F93CF93DF9313
:100BD000EC01688179818A810E943E088C010E9423
:100BE00099070E948A06B801CE010E94BE03DF91D8
:100BF000CF911F910F910895CF93DF93EC019881CE
:100C000089812B813C81232B31F08F3F31F481E0AE
:100C10009F3F19F403C081E001C080E080FD1DC04A
:100C2000CE010E94C201811110C00E94900B882346
:100C3000A1F08A81882389F08091280282FD0DC06D
:100C400082E0DF91CF910C94390CCE010E94E40533
:100C5000CE01DF91CF910C94A301DF91CF91089544
:100C600080E090E00E94161480E090E00E942C1436
:100C70000E94B70B0C94D90B809102019091030153
:100C80000E9488140C9430060E94A70B0C943C061A
:100C900092959F70963079F010F4925001C09A505E
:100CA000923068F4803F69F018F4883E40F409C03F
:100CB000843F29F406C0883E20F0813F11F080E097
:100CC000089581E00895FC01808191810E9433089C
:100CD0000E9448060895CF93DF9300D000D01F9262
:100CE000CDB7DEB70F900F900F900F900F90DF9160
:100CF000CF910895CF93DF9300D000D000D0CDB72F
:100D0000DEB726960FB6F894DEBF0FBECDBFDF91DB
:100D1000CF910895089508950C948B060C948C0639
:100D20000E948E066093AA017093AB018093AC0180
:100D30009093AD010C9430060C9490060F931F9382
:100D40000091AA011091AB012091AC013091AD014D
:100D5000602B712B822B932B1F910F910C9490067B
:100D60000F931F930091AA011091AB012091AC0148
:100D70003091AD0160237123822393231F910F9142
:100D80000C9490060F931F930091AA011091AB0150
:100D90002091AC013091AD01602771278227932704
:100DA0001F910F910C9490060C948B060E94D40610
:100DB0006093A6017093A7018093A8019093A90165
:100DC0000C94300660E070E0CB010C94D6060F93D3
:100DD0001F9341E050E060E070E08A019B0104C095
:100DE000000F111F221F331F8A95D2F7C901B801C6
:100DF0001F910F910C94D6060F931F9341E050E082
:100E000060E070E004C0440F551F661F771F8A958D
:100E1000D2F78091A6019091A701A091A801B0916D
:100E2000A9018A019B01082B192B2A2B3B2BC901F5
:100E3000B8011F910F910C94D6060F931F9341E0B8
:100E400050E060E070E004C0440F551F661F771F3C
:100E50008A95D2F740955095609570958091A6013E
:100E60009091A701A091A801B091A9018A019B01CD
:100E7000082319232A233B23C901B8011F910F918D
:100E80000C94D6060F931F9341E050E060E070E0B1
:100E900004C0440F551F661F771F8A95D2F78091B3
:100EA000A6019091A701A091A801B091A9018A0182
:100EB0009B01082719272A273B27C901B8011F9141
:100EC0000F910C94D6060F931F930091A6011091D9
:100ED000A7012091A8013091A901602B712B822BD1
:100EE000932B1F910F910C94D6060F931F93009193
:100EF000A6011091A7012091A8013091A9016023BA
:100F00007123822393231F910F910C94D6060F9384
:100F10001F930091A6011091A7012091A801309183
:100F2000A90160277127822793271F910F910C94A5
:100F3000D60608952CE0929F800D1124E82FE695A7
:100F4000E695E695877051E001C0550F8A95EAF75E
:100F500085E0E89FF0011124E857FE4F20E030E0E3
:100F600070E04081CB01022E02C0969587950A94CD
:100F7000E2F78170819584278523842781932F5FF1
:100F80003F4F2530310569F708952CE0929F800D81
:100F90001124682F669566956695982F977085E061
:100FA000689FB001112440E050E080E0FB01E40FB5
:100FB000F51FE857FE4F208130E0092E02C036951C
:100FC00027950A94E2F721703327042E01C0220FDF
:100FD0000A94EAF7822B4F5F5F4F4530510531F796
:100FE0000895BF92CF92DF92EF92FF920F931F93DB
:100FF000CF93DF938C01C090A601D090A701E09021
:10100000A801F090A9018091AA019091AB01A09153
:10101000AC01B091AD01C82AD92AEA2AFB2ACFE156
:10102000D0E0D701C6010C2E04C0B695A7959795C0
:1010300087950A94D2F780FD04C0219790F7B12CD0
:1010400007C0BC2EB8018C2F0E94280F0197A9F36E
:101050008B2DDF91CF911F910F91FF90EF90DF903B
:10106000CF90BF900895CF93DF93EC010E94F107DA
:10107000BE010E94280FDF91CF9108951F93CF9357
:10108000DF93EB0190918701992321F0CB010E941E
:10109000330813C0882349F0CB010E94F107182FB1
:1010A000682FCE010E949A0704C0CB010E94C50799
:1010B000182FBE01812F0E94280FDF91CF911F9121
:1010C00008951F93CF93DF93C091AE0116E08091F6
:1010D000AF01C81799F0D0E01C9FF0011D9FF00DE3
:1010E0001124E055FE4F40815181628173818481DA
:1010F00095810E947A062196C770E9CFDF91CF9142
:101100001F9108954091E0015091E1016091E20149
:101110007091E3018091E4019091E5010C947A06CD
:10112000EF92FF920F931F93CF93DF938091E5018E
:1011300082958F7009F065C08091E201882309F4DF
:1011400060C08091AE01F090AF011091E00100917C
:10115000E1016091E3017091E40191E01F3F09F02A
:1011600090E0C0910001D0910101292F96E0E92E75
:101170008F1509F446C06115710521F00F3F21F06C
:1011800030E003C031E001C0322F90E030FD36C0C6
:10119000E89EF001E99EF00D1124DF01A055BE4F3D
:1011A00011963C911197301329C03C91311326C000
:1011B00012963C911297311121C013964D915C917A
:1011C0001497461B570B4C175D07C0F48091E5013F
:1011D0008F7080618093E501EB54FE4F80818F70AA
:1011E0008061808380EE91E00E94FC05DF91CF91C9
:1011F0001F910F91FF90EF900C94610801968770FA
:10120000B7CFDF91CF911F910F91FF90EF9008958D
:101210009F92AF92BF92CF92DF92EF92FF920F9385
:101220001F93CF93DF93CDB7DEB761970FB6F894D6
:10123000DEBF0FBECDBF8C0185E0F801DE011D963B
:1012400001900D928A95E1F7D8011296EC90909159
:10125000E001E091E1012091E3013091E4012115E9
:10126000310531F0EF3F31F481E09F3F19F403C0C5
:1012700081E001C080E0B82FB1709B2E80FD47C196
:10128000D8014C9111965C9111971396AD90BC903A
:10129000149780EEC82E81E0D82EF090E201B501BF
:1012A000621B730B2091000130910101FF2009F4B2
:1012B000D9C08091E5016217730708F095C0282F07
:1012C000207F09F052C05E1313C0491311C0FE2CD9
:1012D000E1100EC08F7080618093E5010E9482084A
:1012E000C6010E94FC058091E501F80185834DC18E
:1012F000AB2831F05F3F31F481E04F3F19F403C078
:1013000081E001C080E080FD03C081E08E2502C045
:1013100080E090E0F82FF170FF2E80FF1CC08091DC
:10132000AE012091AF0136E0821709F40BC190E0C5
:10133000389FF001399FF00D1124E055FE4F618177
:10134000561306C06081461303C06281E61203C0D3
:1013500001968770E9CFFE2CEE2009F416C180912A
:10136000E50181608093E50154C05E1306C0491316
:1013700004C0E11002C0F80199C0C8010E946306D0
:10138000882361F1EE2051F12091E501822F8295B1
:101390008F7090E0029774F08091E0019091E101EC
:1013A00098878F831986BB86AA862C87CE010796DD
:1013B0000E94FC0586E0F801A0EEB1E001900D92DC
:1013C0008A95E1F70E9490080E9482080AC05E1781
:1013D00011F1C8010E94630681112CC0C8010E944E
:1013E000FC05FF24F394D1C0282F207F81F77A2DAC
:1013F000B98AA88A6E2D89890E946B0680EE91E0D9
:101400000E94FC0586E0D6011D928A95E9F70E94AC
:101410008208F12CBAC04913DCCFE110DACFF80111
:101420008583C8010E94FC0586E0D6011D928A953D
:10143000E9F7ABC0EE2091F22091E501822F829571
:101440008F7090E002970CF4B5CF8091E0019091FD
:10145000E1019A8389831B82BD82AC822E83CE01F7
:101460000196A6CF6217730708F044C0FE2CEE2049
:1014700009F4B4CF5E1330C049132EC02091E501AA
:1014800020FD21C0822F82958F70482F50E041159A
:101490005105C9F0F80125834F30510541F08F5FA8
:1014A000982F9295907F822F8F70892B8583C8010A
:1014B0000E94FC0586E0F801A0EEB1E001900D92DB
:1014C0008A95E1F73CC086E0F801A0EEB1E001901A
:1014D0000D928A95E1F759C0C8010E9463068111F7
:1014E00069CF8091E50181608093E501C8010E9488
:1014F000FC054BC07A2DB98AA88A6E2D89890E9475
:101500006B0686E0D6011D928A95E9F718C0EE2099
:1015100009F464CFC8010E946306F82E882309F4F9
:101520005DCF86E0F801A0EEB1E001900D928A95C2
:10153000E1F780EE91E00E9489020E9490080E94EB
:10154000820823C04D875E878D859E850E94330863
:10155000292F22952F70223028F49F7039F08111A5
:1015600005C00BC0243028F49F7049F4805E883099
:1015700020F0C8010E94FC059F2CF92C06C0D80160
:1015800015969C91907F91F7F8CF8F2D61960FB6AD
:10159000F894DEBF0FBECDBFDF91CF911F910F91A9
:1015A000FF90EF90DF90CF90BF90AF909F90089505
:1015B0001F93CF93DF93CDB7DEB72C970FB6F89478
:1015C000DEBF0FBECDBF4F83588769877A878B8771
:1015D0009C87CE0107960E9408098823D1F09F813D
:1015E00088852A853B85232B31F08F3F31F481E0BC
:1015F0009F3F19F403C081E001C080E080FD47C037
:101600004F81588569857A858B859C850E947A06ED
:101610003EC086E0FE013796DE01119601900D92E4
:101620008A95E1F7FF81E8856A857B8561157105FB
:1016300031F0EF3F31F481E0FF3F19F403C081E066
:1016400001C080E080FD23C02091AF0130E0C901DE
:101650000196877099274091AE0150E08417950755
:10166000F1F1F983EA837D836C8396E0929FD00148
:10167000939FB00D1124A055BE4FFE0131960190ED
:101680000D929A95E1F78093AF010E94610816E0F0
:101690008091AE019091AF01891771F1189FC0013F
:1016A000112480559E4F0E940809882329F1E0915A
:1016B000AE011E9FF0011124E055FE4F4081518183
:1016C00062817381848195810E947A068091AE0146
:1016D00090E00196877099278093AE01D9CF0E9440
:1016E00044061092AF011092AE01E0EEF1E086E008
:1016F000DF011D928A95E9F72C960FB6F894DEBFAC
:101700000FBECDBFDF91CF911F9108958091EE0163
:1017100085958595859508958091EE01877008954A
:101720009091EE01977081E009F480E00895809136
:10173000F90108959091F901892B8093F901089599
:1017400080959091F90189238093F9010895109271
:10175000F90108959091F801892B8093F80108957B
:1017600080959091F80189238093F8010895109253
:10177000F80108958091EF01089508950C94BD0B30
:101780000C94BE0B9091280292FD08C09091EF013D
:10179000981721F08093EF010C94C00B089580916D
:1017A000EF01882329F01092EF0180E00C94C00B28
:1017B0000895CF93DF93E0910201F09103018091AE
:1017C000F9018083E0910201F09103019081809101
:1017D000F801892B80838091EF01882381F0E091CB
:1017E0000201F09103019081892B80838091020195
:1017F000909103010E94421481110E94CF0BC0916D
:101800000201D091030148E050E066EE71E0CE01A4
:101810000E943D1C892B69F088E0FE01A6EEB1E034
:1018200001900D928A95E1F7CE01DF91CF910C9452
:101830000B14DF91CF9108950C94BD0B9091280269
:1018400092FD10C098E0899F90011124262B2093CF
:10185000EE010E94FC068091EE01859585958595A7
:101860000C941C0C0C94FC061092EE0180E00C947D
:101870001C0C2091EE01809582238093EE01982F1D
:10188000977099F430E0482F082E000C550B241760
:10189000350759F09091280292FD07C085958595EE
:1018A00085950E941D070C94340C08959091280290
:1018B00092FB222720F9281769F080FB92F9909378
:1018C000280280912702909128020E94A40C82E0B5
:1018D0000C94390C08958091280282FB882780F9A6
:1018E00091E089270C94560C81E00C94560C80E012
:1018F0000C94560C6FEF7FEF80E090E00C94761C18
:1019000080E090E00E94521C21E0893E9E4F09F049
:1019100020E0822F089582E090E00C944A1C83E03E
:1019200090E00C944A1CCF9384E090E00E944A1C03
:10193000C82F82E290E00E944A1C2C2F30E0A901BF
:10194000582BCA01CF910895CF93C92F682F84E0F7
:1019500090E00E94581C6C2F82E290E0CF910C9492
:10196000581CAB01BC018FE090E00C946A1CAB01E9
:10197000BC0183E190E00C946A1C60E070E0CB0154
:101980000C94B70C60E070E0CB010E94B10C0C9499
:10199000BD0C69EE7EEF80E090E00E94761C60E076
:1019A00082E090E00E94581C60E083E090E00E949A
:1019B000581C1092AA011092AB011092AC01109227
:1019C000AD0160E084E090E00E94581C60E082E29B
:1019D00090E00E94581C60E085E090E00E94581C56
:1019E00060E086E090E00E94581C6FEF87E090E096
:1019F0000E94581C40E050E0BA0188E090E00E944C
:101A00006A1C60E08DE090E00E94581C40E050E0CD
:101A1000BA0188E190E00E946A1C60E087E190E0F2
:101A20000E94581C40E050E0BA018CE190E00E9416
:101A30006A1C60E070E080E290E00E94761C40E06A
:101A400050E0BA0188E190E00E946A1C0C94C20C3C
:101A50000C94C90C682F8EE090E00C94581C0E94E6
:101A600037156093060270930702809308029093E3
:101A70000902609302027093030280930402909320
:101A80000502089585B7806885BF85B7806885BFE2
:101A9000089581E008950C94490D08950C944D0D1E
:101AA0000C944D0D0C94500D0C944D0D0C94540D44
:101AB0000C944D0D0E94420D84E090E10E94F513BC
:101AC0000E94580D0C94560D0E944E0D0C944D0D15
:101AD0000E941E100C9423020E9422150E940311E2
:101AE0000E94680D0C94520D5F926F927F928F92BC
:101AF0009F92AF92BF92CF92DF92EF92FF920F939D
:101B00001F93CF93DF93CDB7DEB72A970FB6F89424
:101B1000DEBF0FBECDBF0E941811C82E81110E94DA
:101B20002F0D3AEF832E31E0932E00E010E0502E7F
:101B3000802F0E9442105C01F401619071904F016E
:101B40006826792661147104B1F40F5F1F4F0430C9
:101B5000110569F78FEF89838A831B820E942B15F9
:101B60008160782F9D838C8349815A816B818D811F
:101B70000E943F023AC080910A0281FD0E944B10F0
:101B8000D12CEE24E394F12CC3018E219F21892BCB
:101B900029F10E944B0D8823A9F0DE825F82AE20DE
:101BA000BF2081E0AB2809F480E088870E942B15D4
:101BB0008160782F9A8789874E815F8168858A85C1
:101BC0000E943F02000F111FF801E650FE4F808176
:101BD0009181E826F926F182E08207C0D394EE0CC9
:101BE000FF1CFCE0DF12D0CFB0CF81E0C11001C0FC
:101BF00080E02A960FB6F894DEBF0FBECDBFDF910E
:101C0000CF911F910F91FF90EF90DF90CF90BF90F9
:101C1000AF909F908F907F906F905F9008950E94FB
:101C2000740D0C943402CF93DF930E942D0FEC01BE
:101C3000811522E59207E8F5811531E5930708F053
:101C4000B6C0883E910528F5803E910508F0E9C0B0
:101C5000883A910570F4853A910508F07AC0813090
:101C6000910509F473C008F4D9C0049708F0D9C0ED
:101C7000D5C08F3B910508F0D1C0C85AD0E0CC0F39
:101C8000DD1FCE5BDE4F0990D881C02DCE0194645C
:101C9000C9C0811540E5940708F069C0811550E47A
:101CA000950708F060C09A9581159F4108F4B9C066
:101CB000B5C0811536E5930728F5811545E59407EC
:101CC00008F092C0811554E5950708F087C0AC0173
:101CD00043705527282F26952695C115D34508F022
:101CE0006CC081E090E002C0880F991F4A95E2F72E
:101CF00040E2249F90011124EC01C22BD32BCE0192
:101D00009C6890C081152AE5920780F4811539E519
:101D1000930708F072C0811548E5940708F47EC067
:101D2000D82FCC27CE01806F906A7CC09056811549
:101D3000904208F073C08D2F8F710E94C10FDD2774
:101D4000D0628F71AE01582BCA016CC081E090E067
:101D500069C0C55AD0E0C059DE4F8881C82FD0E095
:101D6000CE0190645FC0DF70CE01906A5BC074E00A
:101D7000969587957A95E1F7282F23703C2F33703D
:101D800081E090E002C0880F991F3A95E2F79C68C5
:101D9000AC01522B9A019C2F9F709695969550E21C
:101DA000959FE0011124C9018C2B9D2B3BC0D82F9E
:101DB000CC27CE01816F906A35C081E090E002C0EF
:101DC000880F991F4A95E2F750E2259F9001112450
:101DD000EC01C22BD32BCE019A6824C0D82FCC277C
:101DE000CE01846F906A1EC00E94C10F8F7190E077
:101DF000D82FCC27CE01906215C08F700E94C10FE2
:101E000094E0D695C7959A95E1F7CF70D0E0DC2F96
:101E1000CC27D0699E01282BC90104C080E090E046
:101E200001C0CE01DF91CF91089520E3829FC001D0
:101E30001124FC012CE0729FE00DF11D1124E60F2E
:101E4000F11DEE0FFF1FE852FF4F85919491089509
:101E50000E94150F0E94130E08958238910569F1B2
:101E6000B0F48133910509F46DC048F489329105CD
:101E700009F463C08A32910509F469C00895853375
:101E8000910509F455C089339105B9F00895833E51
:101E9000910569F138F4803E9105B1F0823E9105DB
:101EA00009F10895863E9105A9F1873E9105B9F1A2
:101EB000843E910509F064C023C02091270220FDD3
:101EC0004FC021FD4DC008958091270280FD44C080
:101ED0008091280280FF44C08091270284FD42C087
:101EE00083EE4DC08091270282FF38C0F5CF8091EC
:101EF000270282FD33C08091280280FD31C0ECCFE3
:101F00008091280281FF32C08091270284FD2AC07F
:101F100087EE35C08091270283FF26C0F5CF8091E0
:101F2000270283FD21C08091280281FD1FC0ECCFD4
:101F30008091270285FD1CC01DC08091270285FD70
:101F400019C016C08091270286FD16C017C0809167
:101F5000270286FD13C010C089E311C082EE0FC0B6
:101F600080EE0DC080E00BC086EE09C084EE07C095
:101F700089E205C085E303C08AE201C081E390E005
:101F800008959091270292FF0DC0282F28712830C4
:101F900019F4877F846006C0282F2471243011F43F
:101FA0008B7F886093FF0DC0282F2871283119F48A
:101FB000877E846106C0282F2471243111F48B7E22
:101FC00088612091280220FF0DC0382F38713830E9
:101FD00019F4877F816006C0382F3171313011F4D8
:101FE0008E7F886021FF0DC0282F2871283119F4B9
:101FF000877E816106C0282F2171213111F48E7EE8
:10200000886194FD877E089580E008950C947A0C91
:102010000E9418118FE39CE90197F1F700C00000BE
:102020000E94181180E00E94421080FF04C00E94AC
:1020300006100C94781508950C9408100E94800CDA
:10204000811102C00E94280D0E948B0C80930A020D
:102050000E94930C90932802809327020E941C10E8
:102060000E948F0C682F70E080E090E00E949C0638
:102070006091A6017091A7018091A8019091A9019A
:102080000C94D406E82FF0E0EE0FFF1FEF5CFD4F3D
:10209000808191810895089580EA8A95F1F70895E5
:1020A00000C008950C944C1008950C9454100C9496
:1020B00055100C9454100C945910F894E82FE29594
:1020C000EF70F0E031A1282F2F7081E090E001C087
:1020D000880F2A95EAF7982F9095932391A392A1C0
:1020E000892B82A3789408950F931F93CF93DF9346
:1020F000CFE7D1E089918F3F11F00E945D1081E020
:10210000C338D807B9F7C3E7D1E00FE711E08991E9
:102110008F3F11F00E945D100C171D07C1F7DF9172
:10212000CF911F910F910895BF92CF92DF92EF92BE
:10213000FF920F931F93CF93DF938C01C62FD0E0B4
:10214000CE0181589E4F6C01FC0190819F3F09F4A4
:1021500050C0B62EF894E92FE295EF70F0E081A11F
:102160009F7021E030E001C0220F9A95EAF7822BA0
:1021700081A382A12095282322A378940E94501045
:10218000E3E7F1E04FE751E021E030E0E12CF12C12
:1021900061916F3F89F0A62FA295AF70B0E0909645
:1021A0008C9190E06F7002C0959587956A95E2F7E3
:1021B00080FD02C0C90102C080E090E0E82AF92A4F
:1021C000220F331F4E175F0719F7F60180818F3FEB
:1021D00011F00E945D1061E0E114F10409F460E087
:1021E0008B2D0E945210CC0FDD1FC00FD11FF98222
:1021F000E882DF91CF911F910F91FF90EF90DF90D8
:10220000CF90BF9008950E94741088E0E1E3F2E05F
:10221000DF01982F1D929A95E9F7E9E2F2E0DF01DC
:102220001D928A95E9F784E00E9463110C94AE0137
:10223000FF920F931F93CF93DF93CDB7DEB728970D
:102240000FB6F894DEBF0FBECDBF8E010F5F1F4FDC
:1022500088E0F80111928A95E9F7F12C6F2DC801F9
:102260000E949410F394F4E0FF12F8CF48E050E09D
:10227000B80189E292E00E943D1CFF24F39400978C
:1022800009F4F12C892B41F088E0F801A9E2B2E0D1
:1022900001900D928A95E1F72F2D44E061E372E001
:1022A00089E292E00E9464110E94B0018F2D28966D
:1022B0000FB6F894DEBF0FBECDBFDF91CF911F9157
:1022C0000F91FF9008950895FF920F931F93CF935E
:1022D000DF93F82E092F162FD72FC42F222349F072
:1022E00081E080930D020E942B1590930C02809345
:1022F0000B0280910D028823D9F080910B029091FE
:102300000C020E944315059798F0EF2DF02FA12F96
:10231000BD2F80E090E04C2F50E08417950734F4F7
:10232000219131912D933D930196F7CF10920D029B
:10233000DF91CF911F910F91FF9008950E94FD169C
:102340000E946C0D0C9409170E940D170E940F0E2D
:102350000C9427170E94C9140E94E4160E945A0D7B
:102360000E949E110E94A4110E94640DFBCFCF9386
:10237000DF93EC01FB018281882309F43CC1C43066
:10238000FDE5DF0760F4CB3F9CE5D90788F49E01AB
:1023900022503C452431310508F02EC109C0C23617
:1023A000EDE5DE0729F0C63AFDE5DF0709F024C1B7
:1023B0000E94930C9093280280932702C1318CE5F0
:1023C000D80709F4C6C008F042C0C930ECE5DE0702
:1023D00009F49BC000F5C5308CE5D80709F485C029
:1023E00078F4C330ECE5DE0709F478C008F07AC071
:1023F000C230DC4509F0F5C0809127028160EFC052
:10240000C7309CE5D90709F478C008F07AC08091FC
:1024100027028061E4C0CD30FCE5DF0709F487C006
:1024200058F4CB309CE5D90709F479C008F07BC09B
:102430008091270288606FC0CF30FCE5DF0709F488
:1024400080C008F082C080912702877FC8C0CE3F3D
:102450009CE5D90709F471C000F5C531FCE5DF073B
:1024600009F485C068F4C3319CE5D90709F475C047
:1024700008F095C00E944406809127028F77AFC074
:10248000CC3FFCE5DF07A9F108F054C0CB3FDC45A9
:1024900009F0A7C08091280240C0C230EDE5DE07F8
:1024A00009F489C058F4C1158DE5D80709F45AC05C
:1024B00008F069C08091280282602FC0C236EDE525
:1024C000DE0709F47CC0C63AFDE5DF0709F481C0E8
:1024D000C330DD4509F085C080E06EC080912702E1
:1024E00082607DC08091270216C08091270288609B
:1024F00076C08091280282604FC08091270280625E
:102500006EC08091270280646AC00E944406809158
:102510002702806864C0846062C081603DC0809191
:1025200027028E7F5CC0809127028D7F58C08091EA
:10253000270216C08091280218C0809128028D7F42
:102540002BC0809127028F7E4AC0809127028F7D09
:1025500046C0809127028F7B42C080912702877FEF
:102560008B7F3DC0809128028D7F8E7F15C080912A
:10257000270282FB222720F991E0922790FB82F923
:1025800090FB83F92CC080912802982F9095917030
:102590008E7F892B90FB81F98093280222C00E94B4
:1025A00044068091270287FB222720F991E0922799
:1025B00090FB87F914C081E00E942A0D12C080911F
:1025C000270284FB222720F991E0922790FB84F9CF
:1025D00006C080912702982F909590FB80F98093F8
:1025E000270280912702909128020E94A40C0E9449
:1025F000440680E001C081E0DF91CF910895CF9340
:10260000DF9386319C4541F5EB010E94970B982F93
:102610008A812091020130910301882379F09A7A0E
:1026200081E009F480E080930E02911102C069E21A
:1026300001C065E3C9010E9484140AC080910E02A2
:10264000811102C069E201C065E3C9010E948614DC
:102650000E94D90B80E001C081E0DF91CF91089505
:102660000F931F93CF93DF93C42FD22FFC0182814E
:102670008823C9F0409311020E942B1590931002F9
:1026800080930F0280E28C0F883008F057C0C7702B
:1026900081E001C0880FCA95EAF7DF91CF911F91C1
:1026A0000F910C94B00380911102481330C08091B7
:1026B0000F02909110020E944315883C910538F555
:1026C00010E21D0FCD17B9F080E28C0F883040F476
:1026D000C77081E001C0880FCA95EAF70E94B7036E
:1026E000183028F581E09D2F977001C0880F9A95CA
:1026F000EAF70E94B003802F0E94A7031830F0F47D
:10270000D77081E001C0880FDA95EAF70AC080E24D
:102710008C0F883098F4C77081E001C0880FCA958B
:10272000EAF7DF91CF911F910F910C94B703802F9F
:10273000DF91CF911F910F910C94A703DF91CF915F
:102740001F910F9108950F939C01CB01243F4CE5FD
:10275000340731F188F4293DFCE53F07D9F02A3DE3
:102760004CE5340779F1283D3C45A9F506E221EE18
:1027700041EE68ED7CE52BC0263FFCE53F07E1F02C
:10278000A8F0273F3C4539F507E225EE46EE67EF16
:102790007CE51DC007E225EE45EE69ED7CE517C03E
:1027A00006E221EE40EE64EF7CE511C007E225EE83
:1027B00044EE65EF7CE50BC006E221EE42EE66EFEB
:1027C0007CE505C008E221E045EE6AED7CE50E946B
:1027D000301380E008C0FC018281882319F0109238
:1027E000110201C081E00F910895909385018093BB
:1027F0008401089590931702809316020895E09142
:102800001602F0911702309721F00190F081E02D2F
:10281000099480E00895E0911602F0911702309734
:1028200021F00280F381E02D099408952091140293
:10283000309115022817390771F090931502809393
:102840001402E0911602F0911702309721F00680F1
:10285000F781E02D0994089520911202309113021E
:102860002817390771F09093130280931202E091B8
:102870001602F0911702309721F00084F185E02DC7
:1028800009940895FC01329697E080E0915029F078
:1028900021912223D9F38F5FF9CF0895662349F060
:1028A000FC01329608962191621729F0E817F90782
:1028B000D1F780E0089581E008959C01FC013296F3
:1028C0009FEF80E04191461789F09F3F19F4411135
:1028D00001C0982F8F5F8630A9F79F3F39F0F9012B
:1028E000E90FF11D97FDFA956283089508959C0103
:1028F0002A5F3F4FFC014281461301C012820196BC
:1029000082179307B9F708950C945D140C9477140B
:10291000029626E0FC0111922A95E9F708950895A0
:102920000C948F1483E0809318020C9490148111FE
:1029300002C081E001C082E0809318020C949014E0
:102940000C94971481E0809318020C9490140C94CA
:10295000A21408950C94A9140C94AA140C94A9140C
:102960000C94A9140C94A914CF930E94B0140E9443
:1029700018110E94AE14C0E08C2F0E944210892BC7
:1029800029F4CF5FC430C1F780E001C081E0CF916E
:10299000089508951F920F920FB60F9211248F93EE
:1029A0009F93AF93BF9380911902811113C08091BF
:1029B000390290913A02A0913B02B0913C024196BB
:1029C000A11DB11D8093390290933A02A0933B025E
:1029D000B0933C02BF91AF919F918F910F900FBE2A
:1029E0000F901F90189580914102843031F10E9420
:1029F00014021092190220E488E190E00FB6F894D6
:102A0000A895809360000FBE2093600083B7817FFC
:102A1000846083BF83B7816083BF7894889583B7D0
:102A20008E7F83BF0FB6F894A8958091600088616F
:102A300080936000109260000FBE08950E944406CB
:102A40000C94180282E084BD93E095BD9AEF97BD87
:102A500080936E0008952FB7F89480913902909179
:102A60003A02A0913B02B0913C022FBF08952FB7CC
:102A7000F8946091390270913A0280913B029091F2
:102A80003C022FBF08959C014FB7F8948091390202
:102A900090913A02A0913B02B0913C024FBF821B41
:102AA000930B089578941F920F920FB60F921124F2
:102AB0008F939F93AF93BF938091390290913A0285
:102AC000A0913B02B0913C020196A11DB11D8093E3
:102AD000390290933A02A0933B02B0933C02BF911B
:102AE000AF919F918F910F900FBE0F901F901895EF
:102AF00087E797E790930108809300089AE088E1C0
:102B00000FB6F894A895809360000FBE9093600074
:102B1000FFCF8091250208950895CF93DF9321E0A0
:102B20002093E9002FEF3091E800215035FD06C0D9
:102B300035ED3A95F1F700002111F5CF2091E8002D
:102B400025FF14C0EC0140E050E068E070E00E9416
:102B500099178091E8008E778093E80088E0FE0165
:102B6000ADE1B2E001900D928A95E1F7DF91CF914E
:102B7000089580931A0270931C0260931B02809147
:102B80004102843001F582E08093E9008FEF90915B
:102B9000E800815095FD06C095ED9A95F1F700008B
:102BA0008111F5CF8091E80085FF0DC040E050E035
:102BB00063E070E08AE192E00E9499178091E8005A
:102BC0008E778093E8000895BC0184E00C94B915D9
:102BD000BC0183E00C94B9150895809140028111E5
:102BE00009C00E942A190E9487198091E20084601E
:102BF0008093E20008951092400208950C94A71467
:102C000060913D0281E0611101C080E00C9492145A
:102C10009091410281E0943009F080E060913D02A2
:102C20000C94971442E061EC81E00E94A31842E208
:102C300061EC82E00E94A3189091410281E09430FF
:102C400009F080E060913D020C94A0148091430251
:102C5000833009F461C030F4813071F0823009F4BE
:102C60009AC008958A3009F486C08B3009F46CC08C
:102C7000893009F0A8C020C080914202813A09F051
:102C8000A2C08091E800877F8093E800809146028F
:102C900090914702892B21F468E08DE192E003C016
:102CA00060E080E090E070E00E94E4178091E8002E
:102CB0008B778093E800089580914202813209F079
:102CC00082C08091460290914702029708F07BC033
:102CD0008091E800877F8093E8008091E80082FD82
:102CE00005C0809141028111F8CF6DC02091F300A1
:102CF0008091F20090E0922B029731F48091F100E4
:102D0000813011F0863021F48091F100809325020A
:102D10008091E8008B7753C080914202813A09F09C
:102D200052C08091460290914702892B09F04BC016
:102D30008091E800877F8093E8008091E80080FF21
:102D4000FCCF8091100136C0809142028132D9F5CA
:102D50008091460290914702892BA9F58091E80065
:102D6000877F8093E8000E94D81880914402809366
:102D700010010C94440680914202813221F5809129
:102D8000E800877F8093E8000E94D8188091450270
:102D900080932602089580914202813AA1F48091A5
:102DA000E800877F8093E8008091E80080FFFCCFF7
:102DB000809126028093F1008091E8008E778093C5
:102DC000E8000C94D818089584B7877F84BF0FB6A5
:102DD000F894A895809160008861809360001092BB
:102DE00060000FBE90E080E80FB6F8948093610019
:102DF000909361000FBE0C94A2140E942A190E94A5
:102E00008719E2EEF0E080818460808378940C94EE
:102E10001C1C84E091E00C94FA13809141028530EF
:102E2000A9F480914102853079F40E94F3148091D5
:102E30003F028823B1F30E94B414882391F30E94C7
:102E400083170E944406EDCF0C941E150895089533
:102E50000C942A17292F332723303105C9F060F449
:102E60002130310581F02230310509F044C08BE377
:102E700090E02AEB31E043C021323105E1F022320B
:102E8000310549F138C082E190E025EF31E037C0EB
:102E900099278130910549F028F0029761F5E8E91A
:102EA000F1E005C0E6EBF1E002C0E8EAF1E0849170
:102EB00090E09F0124C06115710541F061307105FA
:102EC000D1F489E090E025EE31E019C089E090E08E
:102ED0002CEC31E014C06115710541F061307105D1
:102EE00051F482E390E027E032E009C080E490E012
:102EF00029E332E004C080E090E020E030E0FA0115
:102F000031832083089580E189BD82E189BD09B4C0
:102F100000FEFDCF8091D8008F7D8093D8008091F6
:102F2000E00082608093E0008091E00081FDFCCFB2
:102F30000895CF92DF92EF92FF920F931F93CF935A
:102F4000DF93EC018B017A010E94F718811133C0E5
:102F5000E114F10439F0F70180819181081B190B0C
:102F6000C80FD91FC12CD12C0115110519F1809161
:102F7000E80085FD16C08091E8008E778093E80018
:102F8000E114F10449F0F70180819181C80ED91E46
:102F9000D182C08285E00FC00E94F718882321F3F8
:102FA0000AC089918093F10001501109FFEFCF1AF7
:102FB000DF0ADACF80E0DF91CF911F910F91FF9070
:102FC000EF90DF90CF900895209148023091490210
:102FD0002617370748F06115710539F42091E8008C
:102FE0002E772093E80001C0B901FC0120E06115B3
:102FF000710579F1809141028823F1F18530F1F179
:103000008091E80083FD3CC08091E80082FD2EC0E5
:103010008091E80080FFEBCF2091F3008091F200D7
:1030200090E0922B6115710551F08830910538F4CC
:1030300021912093F100615071090196F3CF21E0B5
:10304000089709F020E08091E8008E778093E800EF
:10305000CECF2111CFCF0AC080914102882361F0E9
:10306000853061F08091E80083FD0AC08091E8001E
:1030700082FFF2CF80E0089582E0089583E0089512
:1030800081E00895209148023091490226173707C0
:1030900048F06115710539F42091E8002E772093EE
:1030A000E80001C0B901FC0120E06115710591F152
:1030B00080914102882309F440C0853009F43FC063
:1030C0008091E80083FD3DC08091E80082FD2FC023
:1030D0008091E80080FFE9CF2091F3008091F20019
:1030E00090E0922B6115710559F08830910540F4FC
:1030F00024912093F1003196615071090196F2CF2D
:1031000021E0089709F020E08091E8008E77809315
:10311000E800CBCF2111CCCF0AC080914102882397
:1031200061F0853061F08091E80083FD0AC08091F4
:10313000E80082FFF2CF80E0089582E0089583E006
:10314000089581E00895982F973068F59093E900ED
:10315000981739F07091EC002091ED005091F0003B
:1031600003C0242F762F50E021FD02C09F5FECCFDB
:103170003091EB003E7F3093EB003091ED003D7FCE
:103180003093ED003091EB0031603093EB007093A1
:10319000EC002093ED005093F0002091EE0027FD0D
:1031A000E5CF80E008958F708093E90081E0089575
:1031B0008091420287FF11C08091E80082FD05C026
:1031C000809141028111F8CF11C08091E8008B7786
:1031D0000BC080914102882349F08091E80080FF74
:1031E000F8CF8091E8008E778093E80008952091D1
:1031F000E4003091E50095E64091EC00842F817069
:1032000040FF23C08091E80080FD1DC080914102F5
:10321000882399F0853099F08091EB0085FD11C0ED
:103220004091E4005091E5002417350729F39150AF
:1032300011F09A01E1CF84E0089582E0089583E0DF
:10324000089581E0089580E008954091E80042FFEC
:10325000DDCF08950E9498190E94A019E0EEF0E0D9
:10326000808181608083E8EDF0E080818F778083CA
:1032700019BCA7EDB0E08C918E7F8C9380818F7EFE
:1032800080831092400208950F931F93CF93DF9392
:103290000E9498190E94A019C8EDD0E088818F770C
:1032A000888388818068888388818F7D888319BC22
:1032B0001092410210923D0210923F0210923E0283
:1032C00000EE10E0F80180818B7F8083888181602F
:1032D000888342E060E080E00E94A318E1EEF0E025
:1032E00080818E7F8083E2EEF0E080818160808348
:1032F000808188608083F80180818E7F80838881CF
:1033000080618883DF91CF911F910F910895E8ED3F
:10331000F0E080818F7E8083E7EDF0E08081816046
:10332000808384E082BF81E0809340020C94441942
:10333000E8EDF0E080818E7F80831092E2000895B6
:103340001092DA001092E10008951F920F920FB6CA
:103350000F9211242F933F934F935F936F937F931B
:103360008F939F93AF93BF93EF93FF938091E1006F
:1033700082FF0BC08091E20082FF07C08091E100D4
:103380008B7F8093E1000E941B1C8091DA0080FFFC
:103390001FC08091D80080FF1BC08091DA008E7F13
:1033A0008093DA008091D90080FF0DC080E189BD53
:1033B00082E189BD09B400FEFDCF81E08093410226
:1033C0000E94ED1505C019BC109241020E94FB1528
:1033D0008091E10080FF19C08091E20080FF15C05C
:1033E0008091E2008E7F8093E2008091E200806114
:1033F0008093E2008091D80080628093D80019BC4D
:1034000085E0809341020E9400168091E10084FFD4
:1034100030C08091E20084FF2CC080E189BD82E150
:1034200089BD09B400FEFDCF8091D8008F7D8093C7
:10343000D8008091E1008F7E8093E1008091E200CE
:103440008F7E8093E2008091E20081608093E200B1
:1034500080913D02882311F084E007C08091E30051
:1034600087FD02C081E001C083E0809341020E9499
:1034700008168091E10083FF29C08091E20083FF5C
:1034800025C08091E100877F8093E10082E08093F6
:10349000410210923D028091E1008E7F8093E10015
:1034A0008091E2008E7F8093E2008091E200806153
:1034B0008093E20042E060E080E00E94A3188091E7
:1034C000F00088608093F0000E94FE15FF91EF915C
:1034D000BF91AF919F918F917F916F915F914F912C
:1034E0003F912F910F900FBE0F901F9018951F9234
:1034F0000F920FB60F9211242F933F934F935F9328
:103500006F937F938F939F93AF93BF93CF93DF93EB
:10351000EF93FF93C091E900CF708091EC00D82F1A
:10352000D17080FDD0E81092E9008091F000877F93
:103530008093F00078940E94BB1A1092E900809169
:10354000F00088608093F000CD2BCF70C093E9002D
:10355000FF91EF91DF91CF91BF91AF919F918F91AB
:103560007F916F915F914F913F912F910F900FBE7F
:103570000F901F9018951F93CF93DF93CDB7DEB7B1
:10358000AA970FB6F894DEBF0FBECDBFE2E4F2E01B
:103590008091F100819322E0EA34F207C9F70E949A
:1035A00026168091E80083FF2EC1809142029091FF
:1035B0004302492F50E04A30510508F024C1FA0176
:1035C000EE59FF4F0C94371C803821F0823809F0F7
:1035D0001AC108C080913E0290913F02992389F060
:1035E00082600FC0809146028F70873008F00BC157
:1035F0008093E9008091EB0085FB882780F9109289
:10360000E9009091E800977F9093E8008093F100A3
:103610001092F100D1C0282F2D7F09F0F4C088232B
:1036200019F0823061F0EFC080914402813009F0DE
:10363000EAC0933009F080E080933F022EC0809171
:10364000440281112AC0809146028F702FEF280F0B
:10365000263008F0D8C08093E9002091EB0020FFCD
:103660001CC0933021F48091EB00806214C09091D3
:10367000EB0090619093EB0021E030E0A90102C0E3
:10368000440F551F8A95E2F74093EA001092EA0032
:103690008091EB0088608093EB001092E9008091AC
:1036A000E800877F8093E8000E94D818ACC08111A1
:1036B000AAC0109144021F778091E3008078812B8B
:1036C0008093E3008091E800877F8093E8000E9468
:1036D000D8188091E80080FFFCCF8091E3008068DB
:1036E0008093E300111102C082E001C083E0809367
:1036F000410289C08058823008F085C08091440220
:10370000909145028C3D53E0950779F583E08A83DB
:103710008AE289834FB7F894DE01139620E03EE0F9
:1037200051E2E32FF0E050935700E49120FF03C0F3
:10373000E295EF703F5FEF708E2F90E0EA3010F06F
:10374000C79601C0C0968D939D932F5F243149F792
:103750004FBF8091E800877F8093E8006AE270E0C5
:10376000CE0101960E94E41716C060914602709146
:103770004702AE014F5F5F4F0E942817BC01892BA3
:1037800009F441C09091E800977F9093E800898107
:103790009A810E9442188091E8008B778093E8001C
:1037A00032C0803881F58091E800877F8093E800FF
:1037B00080913D028093F1008091E8008E7772CF76
:1037C000811121C08091440290914502992702976E
:1037D000D4F48091E800877F8093E80080914402D0
:1037E00080933D020E94D81880913D02811106C04D
:1037F0008091E30087FD02C081E001C084E08093F6
:1038000041020E9412168091E80083FF0AC0809155
:10381000E800877F8093E8008091EB0080628093CE
:10382000EB00AA960FB6F894DEBF0FBECDBFDF91B6
:10383000CF911F9108950895CF93809141028823DD
:10384000A1F0C091E900CF709091EC00892F8170B8
:1038500090FD80E8C82B1092E9008091E80083FD7C
:103860000E94BB1ACF70C093E900CF910895EE0F6C
:10387000FF1F0590F491E02D0994FB01DC0104C0C9
:103880008D910190801921F441505040C8F7881B58
:10389000990B0895F999FECF92BD81BDF89A9927A9
:1038A00080B50895A8E1B0E042E050E00C947E1CA1
:1038B000262FF999FECF92BD81BDF89A019700B4E9
:1038C000021639F01FBA20BD0FB6F894FA9AF99A89
:1038D0000FBE08950396272F0E94591C0E94581C62
:1038E000252F0E94591C242F0C94591C0196272F18
:1038F0000E94591C0C94581CDC01CB01FC01F99965
:10390000FECF06C0F2BDE1BDF89A319600B40D922B
:0C39100041505040B8F70895F894FFCFE4
:10391C00C800F00189158D15EC15E815E4158C150A
:10392C0001E200E900EA00B500B600B700CD008363
:10393C0001CC008A01920194012102230224022568
:10394C0002260227022A02B300B4006F0070008125
:10395C008283E200E900EA00B500B600B700CD00B2
:10396C008301CC008A0192019401210223022402DA
:10397C002502260227022A02B300B4006F00700051
:10398C008182839190946697C6343531333236F503
:04399C009293F4000E
:00000001FF
